:100000000C9431080C9475080C9475080C947508C0
:100010000C9475080C9475080C9475080C9475086C
:100020000C9475080C9475080C944C120C941E13C7
:100030000C945B220C9475080C9475080C9475084C
:100040000C9475080C9475080C9475080C9475083C
:100050000C9475080C94C8220C9475080C947508BF
:100060000C9475080C9475080C9475080C9475081C
:100070000C9475080C9475080C9475080C9475080C
:100080000C9475080C9475080C9475080C947508FC
:100090000C9475080C9475080C9475080C947508EC
:1000A0000C9475080C9475080C947508DB2B032CC4
:1000B000042AE12CE12C902BE12CE12C2D2CE12CBD
:1000C000402CAE2CE12CE12CE12CE12C832C6A2C71
:1000D000E12C532CE12C132CE12CE12CDB2CDB2C20
:1000E000DB2CDB2CDB2CDB2CDB2CDB2CDB2CD92CDA
:1000F000E12CD92CE12CE12CE12CE12CE12CE12CA0
:10010000E12CE12CE12CE12CE12CD92CE12CE12C8F
:10011000902B712BDD2CDD2CDD2CDD2CDD2CDD2C52
:10012000DD2CDD2CDD2CDD2CDD2CDD2CBE2CE12CA2
:10013000EF2B626F756E6365213A200025303258CF
:10014000000A000A722F63203031323334353637DB
:1001500038394142434445460A0025303258003A76
:1001600020002530313662000A000000F1A2F1A320
:10017000018C028C35001E001F002000210022008F
:10018000230024002500260027002D002E002A0031
:100190004C002B0014001A000800150017001C006A
:1001A00018000C00120013002F00300031004C002A
:1001B000290004001600070009000A000B000D00CA
:1001C0000E000F0033003400280028004B00E1002F
:1001D0001D001B000600190005001100100036006C
:1001E00037003800E500E50052004E001340E00003
:1001F000E200E300E3002C002C00E700E700E6004B
:10020000E4001340500051004F0001090209005B57
:10021000435D005B445D005B525D005B535D005BD2
:10022000575D0055534220636F6E6669677572654E
:10023000642E0A004B6579626F6172642073746189
:1002400072742E0A005B735D000E03410074006F30
:10025000006D006900630000002C034F0072007401
:100260000068006F006C0069006E0065006100723C
:100270000020004B006500790062006F0061007291
:10028000006400730000000403090409028D0005E6
:100290000100A0FA09040000010301010009211175
:1002A000010001223F000705810308000A0904013B
:1002B000000103010200092111010001224D000784
:1002C00005820308000A0904020001030000000976
:1002D00021110100012236000705830308000A09E5
:1002E0000403000203000000092111010001222083
:1002F000000705840320000107050403200001090D
:100300000404000103000000092111010001223949
:10031000000705850310000112011001000000080C
:10032000EDFE606001000102000105010906A10166
:10033000050719E029E715002501950875018102D7
:1003400005081901290595057501910295017503A7
:100350009101050719002977150025019578750188
:100360008102C00631FF0974A1010975150025FF3E
:100370009520750881020976150025FF95207508DE
:100380009102C005010980A101850216010026B76E
:10039000001A01002AB700751095018100C0050CF4
:1003A0000901A1018503160100269C021A01002AF9
:1003B0009C02751095018100C005010902A1010987
:1003C00001A10005091901290515002501950575EB
:1003D000018102950175038101050109300931157B
:1003E00081257F95027508810609381581257F953D
:1003F0000175088106050C0A38021581257F9501D3
:1004000075088106C0C005010906A101050719E0AC
:1004100029E71500250195087501810295017508E8
:1004200081010508190129059505750191029501BC
:10043000750391010507190029FF150025FF950691
:1004400075088100C06B6579626F6172645F726567
:10045000706F72743A20002530325820000A006B09
:100460006579626F6172645F7365745F6C65643A2D
:10047000200025303258000A006164645F6B6579A2
:100480005F6269743A2063616E2774206164643A24
:1004900020253032580A0064656C5F6B65795F62B5
:1004A00069743A2063616E27742064656C3A202574
:1004B0003032580A00626F6F676D6167696320733D
:1004C00063616E3A202E2E2E2000646F6E652E0A18
:1004D000006D6F7573656B6579205B62746E7C78F7
:1004E0002079207620685D287265702F61636C2901
:1004F0003A205B0025303258007C00256400200043
:10050000256400200025640020002564005D28008B
:100510002575002F00257500290A006565636F6E3B
:100520006669673A0A004C6F636B65642E0A005572
:100530006E6C6F636B65642E0A000A456E7465729B
:1005400020436F6E736F6C65204D6F64650A0043C6
:100550003E20000A0A4A756D7020746F20626F6F2A
:10056000746C6F616465722E2E2E20006E6F742085
:10057000737570706F727465642E0A000A44454288
:1005800055473A2064697361626C65642E0A000AFB
:1005900044454255473A20656E61626C65642E0A97
:1005A000000A44454255473A206D617472697820CB
:1005B000656E61626C65642E0A000A4445425547C7
:1005C0003A206D61747269782064697361626C6548
:1005D000642E0A000A44454255473A206B65796209
:1005E0006F61726420656E61626C65642E0A000A38
:1005F00044454255473A206B6579626F61726420C9
:1006000064697361626C65642E0A000A4445425550
:10061000473A206D6F75736520656E61626C656425
:100620002E0A000A44454255473A206D6F7573659E
:100630002064697361626C65642E0A000A0A2D2DBC
:100640002D2D2D2056657273696F6E202D2D2D2D49
:100650002D0A00444553433A204120636F6D706179
:100660006374206F7274686F6C696E656172206B61
:100670006579626F6172640A005649443A203078A5
:1006800046454544284F7274686F6C696E656172A7
:10069000204B6579626F6172647329205049443A36
:1006A000203078363036302841746F6D69632920E8
:1006B0005645523A203078303030310A00425549A0
:1006C0004C443A2062383961396364202830313A29
:1006D00035343A333620536570202037203230319C
:1006E00035290A004F5054494F4E533A204C554635
:1006F0004120424F4F544D41474943204D4F5553A0
:10070000454B45592045585452414B455920434F7C
:100710004E534F4C4520434F4D4D414E44204E4B80
:10072000524F20343039360A004743433A20342EA2
:10073000372E32204156522D4C4942433A20312E19
:10074000382E30204156525F415243483A2061765C
:1007500072350A0074696D65725F636F756E743A05
:10076000202530346C580A000A0A2D2D2D2D2D20FD
:10077000537461747573202D2D2D2D2D0A00686F13
:1007800073745F6B6579626F6172645F6C656473CB
:1007900028293A2025580A006B6579626F617264D6
:1007A0005F70726F746F636F6C3A2025580A006B2C
:1007B0006579626F6172645F69646C653A2025587F
:1007C0000A004E4B524F3A20656E61626C65640AB6
:1007D000004E4B524F3A2064697361626C65640A43
:1007E000003F0064656661756C745F6C6179657269
:1007F0003A20002575000A0064656275675F636FC3
:100800006E6669672E7261773A2000253032580093
:100810000A002E656E61626C653A20002575000A3B
:10082000002E6D61747269783A20002575000A0007
:100830002E6B6579626F6172643A20002575000A3B
:10084000002E6D6F7573653A20002575000A006BE8
:1008500065796D61705F636F6E6669672E7261772F
:100860003A200025303258000A002E737761705FFD
:10087000636F6E74726F6C5F636170736C6F636BC8
:100880003A20002575000A002E636170736C6F6357
:100890006B5F746F5F636F6E74726F6C3A200025CC
:1008A00075000A002E737761705F6C616C745F6C09
:1008B0006775693A20002575000A002E737761700C
:1008C0005F72616C745F726775693A20002575000C
:1008D0000A002E6E6F5F6775693A20002575000A61
:1008E000002E737761705F67726176655F65736311
:1008F0003A20002575000A002E737761705F6261EF
:10090000636B736C6173685F6261636B7370616367
:10091000653A20002575000A002E6E6B726F3A2032
:10092000002575000A006261636B6C696768745F1B
:10093000636F6E6669672E7261773A2000253032E8
:1009400058000A002E656E61626C653A20002575BC
:10095000000A002E6C6576656C3A20002575000A49
:10096000000A0A2D2D2D2D2D20436F6D6D616E64B3
:100970002048656C70202D2D2D2D2D0A00633A091D
:10098000656E74657220636F6E736F6C65206D6F3A
:1009900064650A00643A09746F67676C6520646572
:1009A00062756720656E61626C650A00783A097449
:1009B0006F67676C65206D61747269782064656229
:1009C00075670A006B3A09746F67676C65206B6521
:1009D00079626F6172642064656275670A006D3ABE
:1009E00009746F67676C65206D6F7573652064654A
:1009F0006275670A00763A097072696E74206465E0
:100A0000766963652076657273696F6E202620694A
:100A10006E666F0A00743A097072696E74207469A8
:100A20006D657220636F756E740A00733A09707297
:100A3000696E74207374617475730A00653A097085
:100A400072696E7420656570726F6D20636F6E667B
:100A500069670A006E3A09746F67676C65204E4BD0
:100A6000524F0A00302F4631303A09737769746368
:100A70006820746F204C6179657230200A00312F34
:100A800046313A0973776974636820746F204C614A
:100A900079657231200A00322F46323A097377693C
:100AA00074636820746F204C6179657232200A008B
:100AB000332F46333A0973776974636820746F2063
:100AC0004C6179657233200A00342F46343A097339
:100AD000776974636820746F204C61796572342083
:100AE0000A00505363723A09706F77657220646F21
:100AF000776E2F72656D6F74652077616B652D75EC
:100B0000700A00436170733A094C6F636B204B6548
:100B100079626F617264284368696C642050726FF7
:100B20006F66290A00506175733A096A756D702005
:100B3000746F20626F6F746C6F616465720A000A73
:100B40000A2D2D2D2D2D20436F6E736F6C6520485F
:100B5000656C70202D2D2D2D2D0A004553432F71CE
:100B60003A09717569740A006D3A096D6F7573659C
:100B70006B65790A007377697463685F64656661A1
:100B8000756C745F6C617965723A20002575002080
:100B9000746F20002575000A00433E20000A51753D
:100BA000697420436F6E736F6C65204D6F64650AC6
:100BB000000A456E746572204D6F7573656B6579BB
:100BC00020436F6E736F6C650A004D303E003F002E
:100BD0000A0A2D2D2D2D2D204D6F7573656B6579AE
:100BE00020506172616D65746572732048656C7028
:100BF000202D2D2D2D2D0A004553432F713A0971BB
:100C00007569740A00313A0973656C656374206D07
:100C10006B5F64656C6179282A31306D73290A0035
:100C2000323A0973656C656374206D6B5F696E742D
:100C3000657276616C286D73290A00333A09736511
:100C40006C656374206D6B5F6D61785F7370656553
:100C5000640A00343A0973656C656374206D6B5FD8
:100C600074696D655F746F5F6D61780A00353A096C
:100C700073656C656374206D6B5F776865656C5F29
:100C80006D61785F73706565640A00363A09736553
:100C90006C656374206D6B5F776865656C5F746904
:100CA0006D655F746F5F6D61780A00703A097072EC
:100CB000696E7420706172616D65746572730A008B
:100CC000643A097365742064656661756C74207696
:100CD000616C7565730A0075703A09696E637265B7
:100CE00061736520706172616D6574657273282B24
:100CF00031290A00646F776E3A0964656372656131
:100D0000736520706172616D6574657273282D3131
:100D1000290A00706775703A09696E6372656173BC
:100D20006520706172616D6574657273282B313056
:100D3000290A007067646F776E3A096465637265AB
:100D400061736520706172616D6574657273282DC1
:100D50003130290A000A7370656564203D2064659E
:100D60006C7461202A206D61785F73706565642002
:100D70002A2028726570656174202F2074696D6562
:100D80005F746F5F6D6178290A007768657265200E
:100D900064656C74613A20637572736F723D0025EF
:100DA00075002C20776865656C3D002575000A008C
:100DB00053656520687474703A2F2F656E2E7769BD
:100DC0006B6970656469612E6F72672F77696B69F3
:100DD0002F4D6F7573655F6B6579730A000A5175E6
:100DE0006974204D6F7573656B657920436F6E7301
:100DF0006F6C650A00433E200073656C6563746523
:100E00006420706172616D657465723A20002575A9
:100E1000000A007365742064656661756C742076E1
:100E2000616C7565732E0A003F004D002575003E0C
:100E300020000A0A2D2D2D2D2D204D6F7573656B09
:100E4000657920506172616D6574657273202D2D16
:100E50002D2D2D0A00313A206D6B5F64656C617930
:100E6000282A31306D73293A20002575000A003296
:100E70003A206D6B5F696E74657276616C286D7374
:100E8000293A20002575000A00333A206D6B5F6D0A
:100E900061785F73706565643A20002575000A000B
:100EA000343A206D6B5F74696D655F746F5F6D615F
:100EB000783A20002575000A00353A206D6B5F777F
:100EC0006865656C5F6D61785F73706565643A2015
:100ED000002575000A00363A206D6B5F77686565FE
:100EE0006C5F74696D655F746F5F6D61783A200047
:100EF0002575000A006D6B5F64656C6179203D208B
:100F0000002575000A006D6B5F696E74657276610D
:100F10006C203D20002575000A006D6B5F6D6178C7
:100F20005F7370656564203D20002575000A006DC3
:100F30006B5F74696D655F746F5F6D6178203D20D4
:100F4000002575000A006D6B5F776865656C5F6DE5
:100F500061785F7370656564203D20002575000A27
:100F6000006D6B5F776865656C5F74696D655F7454
:100F70006F5F6D6178203D20002575000A006D6B64
:100F80005F64656C6179203D20002575000A006D65
:100F90006B5F696E74657276616C203D200025750B
:100FA000000A006D6B5F6D61785F7370656564202A
:100FB0003D20002575000A006D6B5F74696D655FEB
:100FC000746F5F6D6178203D20002575000A006D0B
:100FD0006B5F776865656C5F6D61785F7370656581
:100FE00064203D20002575000A006D6B5F77686501
:100FF000656C5F74696D655F746F5F6D6178203DCE
:1010000020002575000A006261636B6C6967687473
:1010100020696E6372656173653A2025750A006206
:1010200061636B6C69676874206465637265617382
:10103000653A2025750A006261636B6C69676874A4
:1010400020746F67676C653A2025750A00626163DA
:101050006B6C6967687420737465703A2025750A33
:10106000000011241FBECFEFDAE0DEBFCDBF04B613
:1010700003FE24C08091EA019091EB01A091EC0164
:10108000B091ED018730904BA740B04BB9F410926E
:10109000EA011092EB011092EC011092ED0114BEE6
:1010A00084B7877F84BF88E10FB6F894809360008F
:1010B000109260000FBEE0E0F8E3099511E0A0E0B7
:1010C000B1E0E0E9F1E602C005900D92AA33B10764
:1010D000D9F711E0AAE3B1E001C01D92AA3EB10721
:1010E000E1F70E948F0F0C94C6300C940000FF9320
:1010F000EF93E091C701F091C801309709F009958D
:10110000EF91FF910895FC018591803011F0EFDFA0
:10111000FBCF0895FF27E0E230E247FF0CC0419586
:1011200097FF09C0EDE26095709580959095611DDF
:10113000711D811D911D27FF02C0219530E350E2F2
:10114000AA27660F771F881F991FAA1FA41710F0E0
:10115000A41B63955A95A9F7AA3008F0A95FA05D72
:10116000AF93F395611571058105910541F7ED3256
:1011700011F4EF93F395F21718F43F93F395FBCF27
:101180008F91B5DFFA95E1F70895E991F99185918D
:10119000803021F0853219F0AADFF9CF089520E0E0
:1011A000E89455915532C1F3503311F46894559138
:1011B0005A3348F4505390F3220F022E220F220F7D
:1011C000200D250FF4CF0EF4219589919991533676
:1011D00019F3533729F1533559F1BC018827992761
:1011E000E8945C3621F4899199916894559154362C
:1011F00039F446EF7EF077FF0DC08FEF9FEF0AC006
:1012000055374AE039F0583540E121F0523642E096
:1012100009F00895FF93EF937DDFEF91FF91B7CF32
:10122000FF93EF93FC0181918030B9F360DFFBCF36
:10123000FF93EF9368DFF1CFDF93CF93CDB7DEB7A6
:101240002596A3DFCF91DF91089584B18F7984B97A
:1012500085B1806685B98AB18E7D8AB98BB181628C
:101260008BB93E98469A089585B7806885BF85B743
:10127000806885BF0E94E10C6E9A769A0E942509CB
:1012800084B18E7E84B985B1816185B93F98479AD2
:101290008AB181728AB98BB18E6D8BB980B38C7033
:1012A00080BB81B3836F81BB10923B0110923A01E6
:1012B000109245011092440110923D0110923C01A0
:1012C000109247011092460110923F0110923E0188
:1012D0001092490110924801109241011092400170
:1012E00010924B0110924A01109243011092420158
:1012F00010924D0110924C010895AF92BF92CF927F
:10130000EF92FF920F931F93CF93DF93C4E4D1E04A
:1013100010E001E0A5E0CA2EBCE3EB2EB1E0FB2E0D
:10132000123071F018F4113029F407C0133059F05D
:10133000143061F0509A58980BC0559A5D9808C0C7
:10134000259A2D9805C0269A2E9802C03E9A469856
:1013500080EA8A95F1F78FB18695802780FBAA24D1
:10136000A0F8B12C789B03C020E030E002C022E05E
:1013700030E02A293B29189B03C080E090E002C09E
:1013800084E090E0282B392B86B1992787FD909532
:10139000809590958827990F881F9927F3E0880FEB
:1013A000991FFA95E1F7282B392B7C9B03C080E02D
:1013B00090E002C080E190E0282B392B7D9B03C098
:1013C00080E090E002C080E290E0282B392B7E9BE9
:1013D00003C080E090E002C080E490E0282B392B2D
:1013E0008FB1992787FD9095809590958827990FC3
:1013F000881F99279695982F882797958795282B4A
:10140000392B4C9B03C080E090E002C080E091E06B
:10141000282B392B4E9B03C080E090E002C080E077
:1014200092E0282B392B1C9B03C080E090E002C087
:1014300080E094E0282B392B89B1992787FD90957E
:10144000809590958827990F881F9927982F88272E
:10145000990F990F990F282B392B4B9B03C080E0D4
:1014600090E002C080E090E1282B392B4A9B03C01A
:1014700080E090E002C080E090E2282B392B499B6D
:1014800003C080E090E002C080E090E4282B392B7C
:10149000888199818217930741F13983288380914C
:1014A0000001882301F18091C50180FF04C082E31F
:1014B00091E00E9483088091C50180FF0CC080915B
:1014C00000011F928F93FF92EF920E941C090F90D0
:1014D0000F900F900F908091C50180FF04C081E4B0
:1014E00091E00E948308C09200010E9425091F5FBD
:1014F0002296153009F014CF809100018823A1F1C4
:10150000815080930001882339F08FE99FE0019793
:10151000F1F700C0000028C080914401909145017E
:1015200090933B0180933A0180914601909147014D
:1015300090933D0180933C01809148019091490135
:1015400090933F0180933E0180914A0190914B011D
:10155000909341018093400180914C0190914D0105
:10156000909343018093420181E0DF91CF911F91DD
:101570000F91FF90EF90CF90BF90AF900895E82F1C
:10158000F0E0EE0FFF1FE65CFE4F80819181089531
:10159000CF92DF92EF92FF920F931F93CF93DF933F
:1015A00083E491E00E9483082AE3E22E21E0F22EF8
:1015B000C0E0D0E03AE5C32E31E0D32E02E611E0E0
:1015C000DF93CF93DF92CF920E941C098FE591E0C9
:1015D0000E948308F701819191917F010E94052269
:1015E0009F938F931F930F930E941C0988E691E0AD
:1015F0000E94830821968DB79EB708960FB6F8947F
:101600009EBF0FBE8DBFC530D105D1F6DF91CF9102
:101610001F910F91FF90EF90DF90CF900895089564
:101620000895611107C0FC018281882319F02AE026
:1016300032E002C020E030E0C90108958B3B910503
:1016400068F4883A910530F5853A9105C0F4843004
:10165000910598F4019709F06FC071C0803E910523
:1016600008F46AC0883E910540F09C01205F310972
:101670002031310508F060C05CC09C01A1C0853AF2
:10168000910509F45FC0863A910509F45EC023E82C
:1016900030E496C0883A910509F45AC0893A910518
:1016A00009F459C08A3A910509F458C08B3A91055A
:1016B00009F457C08C3A910509F456C08D3A91054A
:1016C00009F455C0803B910509F454C08E3A910548
:1016D00009F453C08F3A910509F452C0813B91053A
:1016E00009F451C0823B910509F450C0833B910538
:1016F00009F44FC0843B910509F44EC0853B910528
:1017000009F44DC0863B910509F44CC0873B910517
:1017100009F44BC0883B910509F44AC0893B910507
:1017200009F449C08A3B910509F048C02AE236E431
:1017300047C09C01306544C020E030E041C021E05A
:1017400030E03EC021E830E43BC022E830E438C05D
:1017500022EE34E435C029EE34E432C02AEE34E41B
:101760002FC025EB34E42CC026EB34E429C027EB52
:1017700034E426C02CEC34E423C02DEC34E420C047
:1017800023E835E41DC02AE835E41AC022E935E42F
:1017900017C024E935E414C021E236E411C023E285
:1017A00036E40EC024E236E40BC025E236E408C07D
:1017B00026E236E405C027E236E402C020E034E445
:1017C000C901089508959FE0799FF00111249BE4D9
:1017D000899FE00DF11D1124E60FF11DEE0FFF1F93
:1017E000EC58FE4F25913491C9010895880F991F37
:1017F00086519040FC0125913491C9010895880FCC
:10180000991F86599E4FFC0125913491C901089575
:101810000E94E30B9C013A9521153F4108F4CDC08D
:101820009C0130522115304120F49F700E94FF0B23
:10183000C4C09C0130532115304120F49C01332752
:10184000306CBCC09C0130542031310528F49C011F
:101850002F703327346DB2C0803120E4920719F421
:1018600020E031EDABC0813140E4940719F420E071
:1018700030EDA4C0823120E4920719F420E032ED6B
:101880009DC0833140E4940719F420E033ED96C005
:10189000811520E5920711F40C94ED22803E91050C
:1018A000E0F4803C910568F58133910509F474C03A
:1018B00048F48932910509F46AC08A32910509F029
:1018C0007AC074C089339105F9F082389105E1F04E
:1018D0008533910509F06FC050C0833E9105A9F191
:1018E00040F4803E9105C9F0823E910509F063C045
:1018F0001BC0863E910571F1873E910509F05BC0E2
:1019000037C00E94F60B59C02091DA0120FD02C0B9
:1019100021FF51C080EE90E04EC08091DA0180FF3F
:10192000F9CF89E390E047C08091DA0182FF0AC0D5
:101930008091DA0184FF03C080E090E03CC083EE38
:1019400090E039C082EE90E036C08091DA0182FFEB
:10195000EFCFF8CF8091DA0183FF07C08091DA01E1
:1019600084FDEACF87EE90E026C086EE90E023C0AB
:101970008091DA0183FFF2CFF8CF8091DA0185FF01
:1019800003C089E290E017C085E390E014C0809125
:10199000DA0185FDF9CFF5CF8091DA0186FF03C02A
:1019A0008AE290E008C081E390E005C08091DA010E
:1019B00086FDF9CFF5CF0E941E0B9C01C901089549
:1019C0000895279A2F988FEF9FEF90938700809329
:1019D00086008AE08093800089E1809381000C94E6
:1019E000622E81110AC080918000877F80938000E1
:1019F00010928D0010928C00089590918000986054
:101A00009093800021E030E002C0220F331F8A95BE
:101A1000E2F72150310930938D0020938C00089516
:101A200080915F0108959091E001943009F04DC0DC
:101A30009091E9009F702091EC0020FF02C020E807
:101A400001C020E0292B94E09093E9009091EB00F5
:101A500090FF38C09091EE0097FF34C090916001E4
:101A6000992321F09091E80095FF2CC0109260011D
:101A700096E014C03091E001343021F53091EB0054
:101A800035FD20C0915021F481E0809360011AC09F
:101A9000EFE9FFE03197F1F700C000003091E80076
:101AA00035FFE8CF8093F1008091E80085FD05C007
:101AB0008091E8008E778093E8002F702093E900F2
:101AC00080E008952F702093E9008FEF0895CF9361
:101AD000DF9300D01F92CDB7DEB72091E001243014
:101AE00021F523E029839B838A832093E9008FEFEC
:101AF00006C095ED9A95F1F70000882329F09091A2
:101B0000E800815095FFF5CF8091E80085FF0DC07A
:101B100040E050E063E070E0CE0101960E94391091
:101B20008091E8008E778093E8000F900F900F90DF
:101B3000DF91CF910895CF93DF9300D01F92CDB75F
:101B4000DEB72091E001243029F522E029839B8330
:101B50008A8383E08093E9008FEF06C095ED9A9524
:101B6000F1F70000882329F09091E800815095FF5B
:101B7000F5CF8091E80085FF0DC040E050E063E0C4
:101B800070E0CE0101960E9439108091E8008E77B6
:101B90008093E8000F900F900F90DF91CF91089500
:101BA0002091E0012430F9F422E02093E9002FEFA6
:101BB00006C035ED3A95F1F70000222329F0309167
:101BC000E800215035FFF5CF2091E80025FF0BC03C
:101BD00040E050E065E070E00E9439108091E8003C
:101BE0008E778093E8000895CF93DF93EC01809186
:101BF000E001843009F045C080910D018823C9F0CF
:101C000085E08093E9008FEF06C095E19A95F1F7A2
:101C10000000882329F09091E800815095FFF5CFCE
:101C20008091E80085FF2DC040E050E060E170E069
:101C300018C081E08093E9008FEF06C095ED9A957A
:101C4000F1F70000882329F09091E800815095FF7A
:101C5000F5CF8091E80085FF14C040E050E068E0D7
:101C600070E0CE010E9439108091E8008E77809359
:101C7000E80080E1FE01AFE4B1E001900D928A95A9
:101C8000E1F7DF91CF9108958FE092E00E94830801
:101C90008091DF01811109C00E94D1110E942E1292
:101CA0008091E20084608093E200089583E192E0F5
:101CB0000E9483081092DF01089587E192E00C945E
:101CC00083088BE192E00E9483080C94100B8FE153
:101CD00092E00E9483080C9457228091E0018430A6
:101CE00049F58091E9008F709091EC0090FF02C05F
:101CF00090E801C090E0982B84E08093E900809107
:101D0000EB0080FF14C08091EE0087FD03C00FC080
:101D10001092F1008091E80085FDFACF8091E800F3
:101D200080FF05C08091E8008E778093E8009F7067
:101D30009093E900089542E061EC81E00E94471130
:101D400042E061EC82E00E94471142E061EC83E0F6
:101D50000E94471146E261EC84E00E94471142E193
:101D600061EC85E00C9447118091E201833009F425
:101D700056C030F4813071F0823009F0AEC095C0A9
:101D80008A3009F482C08B3009F461C0893009F0CF
:101D9000A4C020C08091E101813A09F09EC08091E9
:101DA000E800877F8093E8008091E5019091E6014B
:101DB000892B21F060E080E090E003C060E18FE4D7
:101DC00091E070E00E9488108091E8008B7780930A
:101DD000E80008958091E101813209F07EC0809190
:101DE000E5019091E601009719F0049709F075C09C
:101DF0008091E800877F8093E80005C08091E00132
:101E0000882309F46AC08091E80082FFF7CF8091AF
:101E1000F10080935F018091E8008B775AC0809138
:101E2000E101813A09F059C08091E5019091E60104
:101E3000892B09F052C08091E800877F8093E800E9
:101E40008091E80080FFFCCF80910C013DC0809123
:101E5000E101813209F041C08091E5019091E601F4
:101E6000892BD9F58091E800877F8093E8000E9454
:101E70007E119091E30181E0911101C080E0809397
:101E80000C0180930D010C94801B8091E101813243
:101E900021F58091E800877F8093E8000E947E1101
:101EA0008091E40180934E0108958091E101813A8F
:101EB000A1F48091E800877F8093E8008091E8009A
:101EC00080FFFCCF80914E018093F1008091E8006B
:101ED0008E778093E8000C947E11089584B7877FF5
:101EE00084BF88E10FB6F894809360001092600080
:101EF0000FBE90E080E80FB6F89480936100909355
:101F000061000FBE0E94D1110E942E12E2EEF0E09D
:101F100080818460808383E19DE00C949B210E94FA
:101F20006E0F789402C00E94CB148091E00184303F
:101F3000D1F783E292E00E9483080E947A1582E042
:101F400091E00E94E81484E392E00E9483080FC0AD
:101F500085E492E00E9483080E941C228091DE01A9
:101F6000882329F00E94422281110E94231080912F
:101F7000E001853069F30E94AA15F9CF292F332794
:101F800023303105B1F04CF42130310509F44DC056
:101F90002230310509F04EC007C02132310541F130
:101FA0002232310591F146C0EDE8F0E08BE892E095
:101FB00045C099278130910569F08230910589F0FB
:101FC000892B09F037C0E7E8F2E0E491F0E087E818
:101FD00092E034C0E9E5F2E0E491F0E089E592E0D6
:101FE0002DC0E9E4F2E0E491F0E089E492E026C05B
:101FF000653000F5E62FF0E0EE0FFF1FEA5EFE4FC2
:1020000080819181E9E0F0E019C0653098F4E62F15
:10201000F0E0DF01AA0FBB1FA05EBE4F8D919C9127
:10202000E65DFE4FE081F0E009C0E2E1F0E088E12A
:1020300093E004C0E0E0F0E080E090E0DA018D930E
:102040009C93CF01089580E189BD82E189BD09B4E7
:1020500000FEFDCF8091D8008F7D8093D8008091C5
:10206000E00082608093E0008091E00081FDFCCF81
:102070000895BF92CF92DF92EF92FF920F931F933A
:10208000CF93DF937C018B01EA010E949F11B82E50
:10209000811133C0209731F028813981021B130B45
:1020A000E20EF31EC12CD12C23C08091E80085FDE7
:1020B00015C08091E8008E778093E800209749F062
:1020C000888199818C0D9D1D9983888325E0B22E8E
:1020D00014C00E949F11882359F00EC0F70181910E
:1020E0007F018093F10001501109FFEFCF1ADF0A41
:1020F00001151105D1F601C0B82E8B2DDF91CF91BE
:102100001F910F91FF90EF90DF90CF90BF900895B7
:102110004091E7015091E8014617570748F06115D3
:10212000710539F44091E8004E774093E80001C012
:10213000BA01FC0140E033C08091E001882309F43A
:1021400042C0853009F441C08091E80083FD39C068
:102150008091E80082FD2FC08091E80080FF1FC0C1
:102160009091F3008091F200392F20E0A901482BD3
:10217000CA0106C041914093F10061507109019676
:102180006115710519F088309105A0F341E00897B9
:1021900009F040E08091E8008E778093E8006115B7
:1021A000710551F64111C8CF06C08091E001882326
:1021B00051F0853051F08091E80082FFF6CF80E049
:1021C000089581E0089582E0089583E008954091A4
:1021D000E7015091E8014617570748F0611571056E
:1021E00039F44091E8004E774093E80001C0BA010D
:1021F000FC0140E034C08091E001882309F443C031
:10220000853009F442C08091E80083FD3AC0809196
:10221000E80082FD30C08091E80080FF20C09091EE
:10222000F3008091F200392F20E0A901482BCA0168
:1022300007C044914093F1003196615071090196B5
:102240006115710519F08830910598F341E0089700
:1022500009F040E08091E8008E778093E8006115F6
:10226000710549F64111C7CF06C08091E00188236E
:1022700051F0853051F08091E80082FFF6CF80E088
:10228000089581E0089582E0089583E00895982FED
:102290002CC09093E900981739F07091EC002091D0
:1022A000ED005091F00003C0242F762F50E021FD67
:1022B00002C09F5F1AC03091EB003E7F3093EB006D
:1022C0003091ED003D7F3093ED003091EB003160B7
:1022D0003093EB007093EC002093ED005093F000EE
:1022E0002091EE0027FDE5CF07C0973090F28F7068
:1022F0008093E90081E0089580E008958091E101F4
:1023000087FD05C08091E80080FF0EC012C080915B
:10231000E80082FD05C08091E0018111F8CF0895A9
:102320008091E8008B7708C08091E0018111EACFAD
:1023300008958091E8008E778093E8000895809159
:10234000E4009091E50045E62091EC0020FD1FC0DF
:1023500023C02091E001222391F0253091F02091BB
:10236000EB0025FD10C02091E4003091E500281716
:10237000390751F34150C90139F784E0089582E0EB
:10238000089583E0089581E0089580E00895209104
:10239000E80020FFDECFF9CF2091E80022FFD9CF5F
:1023A000F4CF0E943F120E944712E0EEF0E08081DD
:1023B00081608083E8EDF0E080818F77808319BCB5
:1023C000A7EDB0E08C918E7F8C9380818F7E80838F
:1023D0001092DF0108950F931F93CF93DF930E9414
:1023E0003F120E944712C8EDD0E088818F77888322
:1023F00088818068888388818F7D888319BC10924A
:10240000E0011092DC011092DE011092DD0100EE7D
:1024100010E0F80180818B7F8083888181608883D0
:1024200042E060E080E00E944711E1EEF0E0808150
:102430008E7F8083E2EEF0E0808181608083808106
:1024400088608083F80180818E7F808388818061AD
:102450008883DF91CF911F910F910895E8EDF0E00F
:1024600080818F7E8083E7EDF0E0808181608083D2
:1024700084E082BF81E08093DF010C94EB11E8EDF2
:10248000F0E080818E7F80831092E20008951092A8
:10249000DA001092E10008951F920F920FB60F928A
:1024A00011242F933F934F935F936F937F938F9359
:1024B0009F93AF93BF93EF93FF938091E10082FFCF
:1024C0000BC08091E20082FF07C08091E1008B7F0A
:1024D0008093E1000E946D0E8091DA0080FF1FC0A2
:1024E0008091D80080FF1BC08091DA008E7F80939E
:1024F000DA008091D90080FF0DC080E189BD82E1C2
:1025000089BD09B400FEFDCF81E08093E0010E9407
:10251000440E05C019BC1092E0010E94560E809135
:10252000E10080FF19C08091E20080FF15C080911A
:10253000E2008E7F8093E2008091E20080618093D0
:10254000E2008091D80080628093D80019BC85E0B9
:102550008093E0010E94610E8091E10084FF30C011
:102560008091E20084FF2CC080E189BD82E189BDB9
:1025700009B400FEFDCF8091D8008F7D8093D800F4
:102580008091E1008F7E8093E1008091E2008F7E58
:102590008093E2008091E20081608093E20080916C
:1025A000DC01882311F084E007C08091E30087FFFD
:1025B00002C083E001C081E08093E0010E94670EC9
:1025C0008091E10083FF29C08091E20083FF25C054
:1025D0008091E100877F8093E10082E08093E001B9
:1025E0001092DC018091E1008E7F8093E100809168
:1025F000E2008E7F8093E2008091E2008061809310
:10260000E20042E060E080E00E9447118091F0002B
:1026100088608093F0000E945D0EFF91EF91BF9162
:10262000AF919F918F917F916F915F914F913F916A
:102630002F910F900FBE0F901F9018951F920F9221
:102640000FB60F9211242F933F934F935F936F9385
:102650007F938F939F93AF93BF93CF93EF93FF930A
:102660008091E9008F709091EC0090FF02C090E89B
:1026700001C090E0C92FC82B1092E9008091F000B2
:10268000877F8093F00078940E9462131092E90093
:102690008091F00088608093F000CF70C093E900D3
:1026A000FF91EF91CF91BF91AF919F918F917F91CA
:1026B0006F915F914F913F912F910F900FBE0F90AF
:1026C0001F9018951F93CF93DF93CDB7DEB7AC97CC
:1026D0000FB6F894DEBF0FBECDBFE1EEF1E0809102
:1026E000F100819321E0E93EF207C9F70E94B40EA0
:1026F0008091E80083FF37C18091E1019091E20170
:10270000953009F488C038F49130B1F170F093300D
:1027100009F029C131C0983009F4F8C0993009F4A2
:1027200004C1963009F01FC19DC0803821F0823865
:1027300009F019C108C08091DD019091DE01992353
:1027400089F082600FC08091E5019091E6018F7061
:1027500099278093E9008091EB0085FB882780F919
:102760001092E9009091E800977F9093E8008093A1
:10277000F1001092F100D5C0882319F0823009F0E1
:10278000F2C08F7121F0823009F0EDC00BC0809152
:10279000E301813009F0E7C0933009F080E08093D5
:1027A000DE012FC08091E30181112BC08091E501F2
:1027B0009091E6018F709927009709F4D4C0809317
:1027C000E9002091EB0020FF1CC02091E2012330A2
:1027D00021F48091EB00806212C09091EB00906137
:1027E0009093EB0021E030E001C0220F8A95EAF7D8
:1027F0002093EA001092EA008091EB0088608093B9
:10280000EB001092E9008091E800877F8093E80058
:102810000E947E11A8C08111A6C08091E301909111
:10282000E4018F779927182F9091E3009078982BE7
:102830009093E3008091E800877F8093E8000E94F6
:102840007E118091E80080FFFCCF8091E3008068DA
:102850008093E300112311F083E001C082E08093B4
:10286000E00181C08058823008F07DC08091E30192
:102870009091E4018C3D23E0920779F583E08A830F
:102880008AE289834FB7F894DE01139620E03EE098
:1028900051E2E32FF0E050935700E49120FF03C092
:1028A000E295EF703F5FEF708E2F90E0EA3010F00E
:1028B000C79601C0C0968D939D932F5F243149F731
:1028C0004FBF8091E800877F8093E8006AE270E064
:1028D000CE0101960E94881013C0AE01455D5F4F86
:1028E0006091E5010E94BE0F0097E9F12091E80098
:1028F000277F2093E800BC018BA59CA50E94E710D0
:102900008091E8008B778093E8002DC0803859F5DE
:102910008091E800877F8093E8008091DC018093BC
:10292000F1008091E8008E7771CF81111CC09091E9
:10293000E3019230C0F48091E800877F8093E80043
:102940009093DC010E947E118091DC01811104C012
:102950008091E30087FF02C084E001C081E08093A2
:10296000E0010E949B0E8091E80083FF0AC08091E5
:10297000E800877F8093E8008091EB00806280937D
:10298000EB00AC960FB6F894DEBF0FBECDBFDF9163
:10299000CF911F910895CF938091E0018823B1F0EA
:1029A0008091E9008F709091EC0090FF02C090E858
:1029B00001C090E0C92FC82B1092E9008091E80077
:1029C00083FD0E946213CF70C093E900CF910895F8
:1029D00090936201809361010895809161019091CB
:1029E00062010895E0916101F0916201309721F058
:1029F0000190F081E02D099480E00895FF920F93FB
:102A00001F93CF93DF938C01E0916101F0916201FC
:102A1000309799F10280F381E02D09958091C501ED
:102A200082FF2BC080FF04C085E494E00E948308ED
:102A3000E80180E1F82E07E514E08091C50180FFF0
:102A40000BC088811F928F931F930F930E941C09C4
:102A50000F900F900F900F90FA942196F110EDCFF8
:102A60008091C50180FF09C08DE594E0DF91CF9191
:102A70001F910F91FF900C948308DF91CF911F91CC
:102A80000F91FF900895E0916101F09162013097FC
:102A900021F00480F581E02D0994089520916301CF
:102AA000309164018217930771F0909364018093D1
:102AB0006301E0916101F0916201309721F006809D
:102AC000F781E02D09940895209165013091660108
:102AD0008217930771F09093660180936501E091EE
:102AE0006101F0916201309721F00084F185E02DC1
:102AF000099408950E9484220E9434090E94582358
:102B00000C94622ECF93C82F8091C50182FF1EC006
:102B100080FF04C08FE594E00E9483088091C50186
:102B200080FF0CC01F92CF9322E734E03F932F9396
:102B30000E941C090F900F900F900F908091C5017B
:102B400080FF04C087E794E00E9483088C2FCF9118
:102B50000C94E00C5F926F927F928F929F92AF9253
:102B6000BF92CF92DF92EF92FF920F931F93CF937A
:102B7000DF93CDB7DEB72A970FB6F894DEBF0FBE4E
:102B8000CDBF0E947D0997E6C92E91E0D92E00E0C5
:102B900010E0AA24A394B12C502E802F0E94BF0ACB
:102BA0003C01F601E190F1906F01E826F926E1146D
:102BB000F10431F40F5F1F4F0530110569F73AC07A
:102BC0008091C50181FD0E94C80A20E030E04501E6
:102BD000022E02C0880C991C0A94E2F7C4018E21CF
:102BE0009F21892B09F12E835F826820792081E063
:102BF000672809F480E088870E948D228160782F01
:102C00009A8789874E815F8168858A850E946316CD
:102C1000F801EE0FFF1FE959FE4F80819181882551
:102C200099259183808316C02F5F3F4F2F30310548
:102C300071F6C0CF8FEF89838A831B820E948D2219
:102C40008160782F9D838C8349815A816B818D812E
:102C50000E9463160E94D626109171010E94F21400
:102C60001817D9F00E94F214809371012A960FB6BA
:102C7000F894DEBF0FBECDBFDF91CF911F910F91B2
:102C8000FF90EF90DF90CF90BF90AF909F908F908C
:102C90007F906F905F900C9482152A960FB6F894EF
:102CA000DEBF0FBECDBFDF91CF911F910F91FF907F
:102CB000EF90DF90CF90BF90AF909F908F907F90DC
:102CC0006F905F900895CF93DF93CDB7DEB72B97CA
:102CD0000FB6F894DEBF0FBECDBF4F83588769870C
:102CE0007A878B87DE01119686E0FD0111928A9525
:102CF000E9F785E0FE01379601900D928A95E1F79C
:102D000049815A816B817C818D819E810E943B1E0D
:102D10002B960FB6F894DEBF0FBECDBFDF91CF91DB
:102D20000895CF93C82F882309F4C1C0823859F47D
:102D30000E94F21481FDBBC089E30E94A0200E9482
:102D4000752189E30CC0833879F40E94F21480FD68
:102D5000AEC083E50E94A0200E94752183E50E94F9
:102D6000EE20CF910C947521843859F40E94F2140E
:102D700082FD9DC087E40E94A0200E94752187E407
:102D8000EECF8450813A48F48C2F0E94EC2C8111B4
:102D90008EC08C2F0E94A020E4CF8C2F805E8830C4
:102DA00050F4C77081E090E001C0880FCA95EAF73F
:102DB0000E943C21D6CF8C2F855A833078F4C53AB7
:102DC00029F0C63A31F482E890E005C081E890E04D
:102DD00002C083E890E0CF910C944E158C2F885A56
:102DE000833108F064C0C83A39F1C93A41F1CA3AAE
:102DF00049F1CB3A51F1CC3A59F1CD3A61F1C03BAE
:102E000069F1CE3A71F1CF3A79F1C13B81F1C23B20
:102E100089F1C33B91F1C43B99F1C53BA1F1C63B9C
:102E2000A9F1C73BB1F1C83BB9F1C93BC1F1CA3BFC
:102E3000C9F58AE292E038C082EE90E035C089EEB2
:102E400090E032C08AEE90E02FC085EB90E02CC07D
:102E500086EB90E029C087EB90E026C08CEC90E0F8
:102E600023C08DEC90E020C083E891E01DC08AE88B
:102E700091E01AC082E991E017C084E991E014C0A2
:102E800081E292E011C083E292E00EC084E292E01F
:102E90000BC085E292E008C086E292E005C087E2BE
:102EA00092E002C080E090E0CF910C946415CF9145
:102EB0000895882309F44DC0823859F40E94F21411
:102EC00081FF47C089E30E94A0200E94752189E309
:102ED0000CC0833871F40E94F21480FF3AC083E57D
:102EE0000E94A0200E94752183E50E94EE200C9490
:102EF0007521843859F40E94F21482FF2AC087E4B5
:102F00000E94A0200E94752187E4EFCF982F945053
:102F1000913A08F4EACF982F905E983058F4282F11
:102F2000277081E090E001C0880F2A95EAF70E949F
:102F30004221DDCF982F955A933020F480E090E025
:102F40000C944E15885A833120F480E090E00C9464
:102F500064150895882321F00E943C210C9475216A
:102F60000895882321F00E9442210C947521089530
:102F7000BF92CF92DF92EF92FF920F931F93CF9366
:102F8000DF93CDB7DEB727970FB6F894DEBF0FBE3D
:102F9000CDBF8C0185E0F801DE01119601900D9204
:102FA0008A95E1F7F80130812181F28055815295AF
:102FB0005F7083819481892B39F02F3F41F481E048
:102FC00090E03F3F31F003C081E090E002C080E03C
:102FD00090E080FD73C339832A8389819A815E835F
:102FE0000E945D20B92E8F830E945C200E94841F66
:102FF0002B2D22952F7030E05E816F8125303105B9
:1030000009F4E6C06CF4243031050CF0A2C04B2D5D
:10301000407F8B2D8F70223031050CF045C017C0DA
:103020002C3031054CF42A3031050CF0E7C1283042
:10303000310509F043C3E5C02D30310509F4BAC2AA
:103040000CF4A2C22F30310509F038C323C3182F66
:10305000411101C002C01295107FFF2059F01123C9
:1030600009F46BC2812F6F830E944C210E9475214D
:103070006F8163C2862F0E945917112309F41EC362
:10308000812F0E94522127960FB6F894DEBF0FBE03
:10309000CDBFDF91CF911F910F91FF90EF90DF9007
:1030A000CF90BF900C947521403211F08295807FB3
:1030B000662319F0613071F523C0FF20B1F0511182
:1030C00001C032C0513081F527960FB6F894DEBFAB
:1030D0000FBECDBFDF91CF911F910F91FF90EF9069
:1030E000DF90CF90BF900C945C21511101C003C0C0
:1030F000513009F4E3C28E830E945F218E819AC110
:10310000FF2021F0563008F0D9C20EC0553008F02B
:10311000D5C290C1FF20C9F0552331F0F801958147
:1031200090FF0BC29F70958327960FB6F894DEBF71
:103130000FBECDBFDF91CF911F910F91FF90EF9008
:10314000DF90CF90BF900C94AA17552309F472C159
:1031500009C22B2D26952695237030E021153105C7
:1031600029F02130310509F0A9C219C0FF2021F052
:10317000862F9B2D937002C080E090E027960FB6BB
:10318000F894DEBF0FBECDBFDF91CF911F910F919D
:10319000FF90EF90DF90CF90BF900C944E15FF20E2
:1031A00021F0862F9B2D937002C080E090E027963F
:1031B0000FB6F894DEBF0FBECDBFDF91CF911F9148
:1031C0000F91FF90EF90DF90CF90BF900C9464151B
:1031D000862FFF2019F00E945A2502C00E94C225A6
:1031E00027960FB6F894DEBF0FBECDBFDF91CF910B
:1031F0001F910F91FF90EF90DF90CF90BF900C94B4
:1032000049268B2D837009F079C0F11057C2262F03
:10321000229526952770220F220F862F8F70C82E99
:10322000D12CE12CF12C022E04C0CC0CDD1CEE1CA8
:10323000FF1C0A94D2F764FF10C06FE070E080E0DA
:1032400090E004C0660F771F881F991F2A95D2F758
:10325000609570958095909503C060E070E0CB011B
:103260002B2D269526952370422F50E04230510594
:10327000D9F04330510569F16C297D298E299F29A8
:103280004130510551F127960FB6F894DEBF0FBEBD
:10329000CDBFDF91CF911F910F91FF90EF90DF9005
:1032A000CF90BF900C94991F6C297D298E299F295E
:1032B00027960FB6F894DEBF0FBECDBFDF91CF913A
:1032C0001F910F91FF90EF90DF90CF90BF900C94E3
:1032D000AB1F0E94991FC701B60127960FB6F8943D
:1032E000DEBF0FBECDBFDF91CF911F910F91FF9039
:1032F000EF90DF90CF90BF900C94871FFF2019F0C4
:103300008B2D817001C08695882309F4D7C1262FA3
:10331000229526952770220F220F862F8F70C82E98
:10332000D12CE12CF12C022E04C0CC0CDD1CEE1CA7
:10333000FF1C0A94D2F764FF10C06FE070E080E0D9
:1033400090E004C0660F771F881F991F2A95D2F757
:10335000609570958095909503C060E070E0CB011A
:103360002B2D269526952370422F50E04230510593
:10337000D9F04330510569F16C297D298E299F29A7
:103380004130510551F127960FB6F894DEBF0FBEBC
:10339000CDBFDF91CF911F910F91FF90EF90DF9004
:1033A000CF90BF900C9438206C297D298E299F29BD
:1033B00027960FB6F894DEBF0FBECDBFDF91CF9139
:1033C0001F910F91FF90EF90DF90CF90BF900C94E2
:1033D0004A200E943820C701B60127960FB6F894FC
:1033E000DEBF0FBECDBFDF91CF911F910F91FF9038
:1033F000EF90DF90CF90BF900C942620603F59F162
:1034000020F4603E08F494C008C0623F09F467C02D
:10341000F0F1633F09F08CC065C0162F1F708B2D33
:103420008F71FF2021F00E94D11F812F7DCE0E943D
:10343000EC1F812F27960FB6F894DEBF0FBECDBFCD
:10344000DF91CF911F910F91FF90EF90DF90CF9080
:10345000BF900C94B117FF20B1F0553008F02EC189
:103460008B2D8F7127960FB6F894DEBF0FBECDBFA0
:10347000DF91CF911F910F91FF90EF90DF90CF9050
:10348000BF900C940B20563008F018C1E9CFFF20F4
:1034900099F08B2D8F7127960FB6F894DEBF0FBE73
:1034A000CDBFDF91CF911F910F91FF90EF90DF90F3
:1034B000CF90BF900C94D11F8B2D8F7127960FB694
:1034C000F894DEBF0FBECDBFDF91CF911F910F915A
:1034D000FF90EF90DF90CF90BF900C94EC1FF11015
:1034E000EBCFD7CFFF2099F08B2D8F7127960FB69A
:1034F000F894DEBF0FBECDBFDF91CF911F910F912A
:10350000FF90EF90DF90CF90BF900C94C21F279652
:103510000FB6F894DEBF0FBECDBFDF91CF911F91E4
:103520000F91FF90EF90DF90CF90BF900C94BD1F54
:10353000FF20A9F0552309F4ACCF862F27960FB6AC
:10354000F894DEBF0FBECDBFDF91CF911F910F91D9
:10355000FF90EF90DF90CF90BF900C949116552381
:1035600009F4AACF862F27960FB6F894DEBF0FBEB8
:10357000CDBFDF91CF911F910F91FF90EF90DF9022
:10358000CF90BF900C9459174B2D4F70C8010E94DB
:10359000110B27960FB6F894DEBF0FBECDBFDF919B
:1035A000CF911F910F91FF90EF90DF90CF90BF9040
:1035B0000C94F11EF11082C09B2D9F70492F50E09A
:1035C0004230510599F144F44115510569F04130FB
:1035D000510509F073C019C043305105C1F14430A1
:1035E000510509F06BC044C027960FB6F894DEBFB2
:1035F0000FBECDBFDF91CF911F910F91FF90EF9044
:10360000DF90CF90BF900C94732E27960FB6F8944E
:10361000DEBF0FBECDBFDF91CF911F910F91FF9005
:10362000EF90DF90CF90BF900C949D2E27960FB611
:10363000F894DEBF0FBECDBFDF91CF911F910F91E8
:10364000FF90EF90DF90CF90BF900C94CC2E2796F8
:103650000FB6F894DEBF0FBECDBFDF91CF911F91A3
:103660000F91FF90EF90DF90CF90BF900C94F22ECF
:10367000862F27960FB6F894DEBF0FBECDBFDF9121
:10368000CF911F910F91FF90EF90DF90CF90BF905F
:103690000C94292F4B2D4F70C80127960FB6F89424
:1036A000DEBF0FBECDBFDF91CF911F910F91FF9075
:1036B000EF90DF90CF90BF900C94E20B27960FB65F
:1036C000F894DEBF0FBECDBFDF91CF911F910F9158
:1036D000FF90EF90DF90CF90BF9008950E94592106
:1036E0000E942E210E9475210E9477270E94492660
:1036F00080E090E00E944E1580E090E00C9464150C
:103700000E9449210C946E1B0E945D20292F229556
:103710002F7030E02C3031054CF42A3031056CF438
:10372000225031092230310570F407C02C303105A8
:1037300031F02F30310539F402C081E0089593FB58
:10374000882780F9089580E00895CF93DF9300D013
:1037500000D01F92CDB7DEB70F900F900F900F9053
:103760000F90DF91CF910895CF93DF9300D000D0D9
:1037700000D0CDB7DEB726960FB6F894DEBF0FBEE9
:10378000CDBFDF91CF9108951F93CF93DF93C09169
:10379000A80116E012C0D0E01C9FF0011D9FF00DA3
:1037A0001124E858FE4F40815181628173818481E8
:1037B00095810E94B41B2196C7708091A901C813FE
:1037C000EACFDF91CF911F910895409172015091FE
:1037D00073016091740170917501809176019091EF
:1037E00077010C94B41B0F931F93CF93DF938091B9
:1037F000770182958F7009F069C0809174018823E8
:1038000009F464C0A091A801D091A901B0917201FE
:10381000C0917301809175019091760121E030E0B3
:10382000BF3F11F020E030E0122FBC016095709591
:1038300006E04AC0009721F0CF3F29F4212F05C0B0
:1038400021E030E002C020E030E020FD3BC04A2F04
:1038500050E0049FF001059FF00D1124E858FE4F41
:103860002181C2132FC02081B2132CC022812111CB
:1038700029C0238134812817390718F0281B390BF8
:1038800002C0260F371F283C3105E0F480917701F4
:103890008F7080618093770186E0849FF001859F1F
:1038A000F00D1124E358FE4F80818F70806180837A
:1038B00082E791E00E94B817DF91CF911F910F919D
:1038C0000C94C41BAF5FA770AD13B4CFDF91CF9141
:1038D0001F910F910895EF92FF920F931F93CF9333
:1038E000DF93CDB7DEB762970FB6F894DEBF0FBE99
:1038F000CDBF8C0185E0F801DE011D9601900D928F
:103900008A95E1F7D8014C9111965C911197129626
:103910006C9112971396ED90FC9014977091720130
:10392000E09173018091750190917601009739F0D3
:10393000EF3F41F421E030E07F3F31F003C021E070
:1039400030E002C020E030E020FD5CC12091740135
:10395000222309F4F1C0E816F90628F09701281B84
:10396000390BC90104C0809590958E0D9F1D883C30
:10397000910508F098C080917701982F907F09F009
:1039800064C0E51314C0741312C0611110C08F70AD
:103990008061809377010E94E51B82E791E00E949D
:1039A000B81780917701D80115968C9343C1EF2801
:1039B00039F05F3F41F481E090E04F3F31F003C0C8
:1039C00081E090E002C080E090E080FD03C081E0F3
:1039D000862702C080E090E080FF2EC08091A80181
:1039E0002091A90136E013C090E0389FF001399F83
:1039F000F00D1124E858FE4F7181571306C07081F5
:103A0000471303C07281671317C001968770821332
:103A1000EBCF12C19F7059F0882309F40BC107C086
:103A20009F7029F0F8019581907F09F403C1805EB1
:103A3000883008F4FFC0D2C0662309F4FBC080912F
:103A40007701816080937701F5C0E51308C0741396
:103A500006C0611104C0D80115968C939DC04D8796
:103A60005E878D859E856A8B0E94841B6A89882368
:103A700009F4B4C0662309F4B1C020917701822F04
:103A800082958F7090E002970CF4C6C0809172010D
:103A90009091730198878F831986FB86EA862C871D
:103AA000CE01079646C080917701982F907F59F4F8
:103AB0007E2DF98AE88A89890E94A51B82E791E018
:103AC0000E94B81795C0E51311C074130FC061119F
:103AD0000DC0F8018583C8010E94B817E2E7F1E044
:103AE00086E0DF011D928A95E9F7A2C04D875E87C7
:103AF0008D859E856A8B0E94841B6A89882309F4C0
:103B00006DC0662309F46AC020917701822F8295E7
:103B10008F7090E002970CF47FC0809172019091B9
:103B200073019A8389831B82FD82EC822E83CE01EE
:103B300001960E94B81770C0E816F90628F09701A0
:103B4000281B390BC90104C0809590958E0D9F1DCF
:103B5000883C910508F046C0662309F43FC0E51390
:103B600030C074132EC02091770120FD21C0322F68
:103B700032953F70832F90E00097D1F0D8011596D1
:103B80002C9315970F9741F0832F8F5F8295807F3D
:103B90002F70282B15962C93C8010E94B81786E029
:103BA000F801A2E7B1E001900D928A95E1F73EC0DD
:103BB00086E0F801A2E7B1E001900D928A95E1F765
:103BC00037C04D875E878D859E850E94841B81113D
:103BD00023C080917701816080937701C8010E94A2
:103BE000B81726C07E2DF98AE88A89890E94A51B0C
:103BF000E2E7F1E086E0DF011D928A95E9F70E9495
:103C0000E51B18C0662351F34D875E878D859E8521
:103C10000E94841B882311F386E0F801A2E7B1E03B
:103C200001900D928A95E1F70E94F31B0E94E51B1B
:103C300081E014C080E012C04D875E878D859E852F
:103C40000E945D20292F22952F7030E0223031050F
:103C50000CF4E0CE243031050CF6E2CE62960FB6BD
:103C6000F894DEBF0FBECDBFDF91CF911F910F91B2
:103C7000FF90EF9008951F93CF93DF93CDB7DEB7FA
:103C80002C970FB6F894DEBF0FBECDBF4F83588779
:103C900069877A878B879C87CE0107960E946B1C69
:103CA0008823D9F02F8138858A859B85892B39F027
:103CB0003F3F19F080E090E004C02F3FD9F781E04A
:103CC00090E0892B09F06DC04F81588569857A8510
:103CD0008B859C850E94B41B64C086E0FE013796EC
:103CE000DE01119601900D928A95E1F7FF81E8853A
:103CF0004A855B854115510539F0EF3F41F481E07C
:103D000090E0FF3F31F003C081E090E002C080E02E
:103D100090E080FD46C02091A90130E0C9010196E4
:103D2000877099276091A80170E08617970709F4BA
:103D300040C0F983EA835D834C8396E0929FD00173
:103D4000939FB00D1124A858BE4FFE0131960190EB
:103D50000D929A95E1F78093A9010E94C41B21C09E
:103D6000189FC001112488589E4F0E946B1C882305
:103D700071F1E091A8011E9FF0011124E858FE4F57
:103D80004081518162817381848195810E94B41B3D
:103D90008091A80190E00196877099278093A801EF
:103DA00001C016E08091A8019091A9018913D8CF94
:103DB0000EC00E94801B1092A9011092A801E2E798
:103DC000F1E086E0DF011D928A95E9F7EACF2C96B3
:103DD0000FB6F894DEBF0FBECDBFDF91CF911F911C
:103DE0000895DF92EF92FF920F931F93CF93DF938B
:103DF000EC01009709F46CC0D12CEE24E394F12C73
:103E00008E010F5F1F4FFE018491843748F4843088
:103E100008F04AC0813071F0823009F059C01EC0EC
:103E2000853709F43DC070F1982F9458903708F009
:103E30004FC03DC02296F8018491982F905E983033
:103E400050F48770FE2D01C0FF0F8A95EAF78F2F7F
:103E50000E944C2130C00E9491162DC02296F8017C
:103E60008491982F905E983050F48770FE2D01C099
:103E7000FF0F8A95EAF78F2F0E9452211CC00E94E3
:103E8000591719C02296F801049107C08FE99FE0E5
:103E90000197F1F700C0000001500111F7CF0BC0EE
:103EA0002296F801D49007C00E94911603C08F7724
:103EB0000E945917E8018D2D07C08150EFE9FFE0FE
:103EC0003197F1F700C00000882309F499CFF5CFAE
:103ED000DF91CF911F910F91FF90EF90DF900895A8
:103EE0006093AE017093AF018093B0019093B101E4
:103EF0000C946E1B6093AA017093AB018093AC018C
:103F00009093AD010C946E1B08950C94701F0F9349
:103F10001F930091AE011091AF012091B00130913B
:103F2000B101602B712B822B932B1F910F910C945D
:103F3000701F0F931F930091AE011091AF0120915C
:103F4000B0013091B10160237123822393231F912B
:103F50000F910C94701F0F931F930091AE0110915D
:103F6000AF012091B0013091B10160277127822704
:103F700093271F910F910C94701F60E070E0CB01AC
:103F80000C947A1F41E050E060E070E004C0440F00
:103F9000551F661F771F8A95D2F7CB01BA010C9483
:103FA0007A1F41E050E060E070E004C0440F551F0C
:103FB000661F771F8A95D2F78091AA019091AB0175
:103FC000A091AC01B091AD01482B592B6A2B7B2BF2
:103FD000CB01BA010C947A1F41E050E060E070E040
:103FE00004C0440F551F661F771F8A95D2F740956E
:103FF0005095609570958091AA019091AB01A09128
:10400000AC01B091AD01482359236A237B23CB0136
:10401000BA010C947A1F41E050E060E070E004C007
:10402000440F551F661F771F8A95D2F78091AA010A
:104030009091AB01A091AC01B091AD0148275927F7
:104040006A277B27CB01BA010C947A1F0F931F9329
:104050000091AA011091AB012091AC013091AD010A
:10406000602B712B822B932B1F910F910C947A1F35
:104070000F931F930091AA011091AB012091AC0105
:104080003091AD0160237123822393231F910F91FF
:104090000C947A1F0F931F930091AA011091AB010A
:1040A0002091AC013091AD016027712782279327C1
:1040B0001F910F910C947A1F0895CF92DF92EF9287
:1040C000FF920F931F93CF93DF93EC01C090AE014B
:1040D000D090AF01E090B001F090B1018091AA01C1
:1040E0009091AB01A091AC01B091AD01C82AD92A41
:1040F000EA2AFB2A0FE110E0B701A601002E04C056
:1041000076956795579547950A94D2F740FF08C072
:10411000BE01802F0E94080C8130910509F007C074
:104120000150110948F7BE0180E00E94080CDF91A0
:10413000CF911F910F91FF90EF90DF90CF90089556
:1041400090910D01992341F1982F9695969596950A
:104150009F3088F4E0910E01F0910F01E90FF11DFD
:10416000877021E030E001C0220F8A95EAF7818153
:10417000822B818308959091C50190FF2EC01F92DC
:104180008F9389E794E09F938F930E941C090F906F
:104190000F900F900F90089540910E0150910F01D4
:1041A00020E030E09FEFFA01E20FF31F6281681711
:1041B000A1F09F3F19F4611101C0922F2F5F3F4F73
:1041C0002E30310581F707C0FA01E90FF11D97FD87
:1041D000FA95828308959F3FB9F7089590910D0154
:1041E000992349F1982F9695969596959F3090F43E
:1041F000E0910E01F0910F01E90FF11D877021E0B0
:1042000030E001C0220F8A95EAF7209581812823AA
:10421000218308959091C50190FF1FC01F928F9335
:1042200087E994E09F938F930E941C090F900F9051
:104230000F900F90089540910E0150910F0120E0D2
:1042400030E0FA01E20FF31F9281981301C012824D
:104250002F5F3F4F2E303105A1F7089581E090E0A8
:10426000E0910E01F0910F01E80FF91F1082019605
:1042700080319105A9F708959091B201982B909300
:10428000B201089580959091B20198239093B20164
:1042900008951092B20108959091B301982B9093D4
:1042A000B301089580959091B30198239093B30141
:1042B00008951092B30108958093B4010895109267
:1042C000B401089540910E0150910F0120E030E0BB
:1042D00080E0FA01E20FF31F918191118F5F2F5F50
:1042E0003F4F2F303105A9F70895E0910E01F0916D
:1042F0000F018091B2018083E0910E01F0910F01D6
:1043000080819091B301892B80839091B40199238E
:1043100061F0E0910E01F0910F018081892B808383
:104320000E94622181110E945F2180910E01909173
:104330000F010C94FE149093C8018093C701089557
:10434000CF92DF92EF92FF920F931F936C01EE24B6
:10435000FF24C114D104E104F10421F46B017C01B8
:1043600080E001C080E133272F2D1E2D0D2D01157A
:1043700011052105310519F0885F68017901970160
:104380008601A4E03695279517950795AA95D1F74C
:10439000011511052105310519F08C5F68017901BE
:1043A00097018601F2E03695279517950795FA95BE
:1043B000D1F7011511052105310519F08E5F68014E
:1043C0007901B701A6017695679557954795452BD5
:1043D000462B472B09F08F5F1F910F91FF90EF90B5
:1043E000DF90CF9008958295982F9C7C9695969516
:1043F000837344E0849F90011124922B892F8A7A41
:1044000086959575990F892B08951F93CF93DF9308
:104410001F92CDB7DEB799830E94F321182F99819F
:10442000892F0E94F321312F20E0282BC9010F9002
:10443000DF91CF911F9108958091E001843009F1BF
:104440001092C60120E488E190E00FB6F894A89598
:10445000809360000FBE2093600083B7817F8460EB
:1044600083BF83B7816083BF7894889583B78E7F3D
:1044700083BF88E10FB6F8948093600010926000CB
:104480000FBE0895CF930E940F0B0E947D090E94DA
:10449000100BC0E08C2F0E94BF0A892B29F4CF5F3C
:1044A000C530C1F780E001C081E0CF9108950E943E
:1044B000801B0C94622E1F920F920FB60F92112444
:1044C0008F939F93AF93BF938091C601811113C0C7
:1044D0008091C9019091CA01A091CB01B091CC010A
:1044E0004196A11DB11D8093C9019093CA01A0936B
:1044F000CB01B093CC01BF91AF919F918F910F9061
:104500000FBE0F901F90189582E084BD93E095BD7B
:104510009AEF97BD80936E0008958FB7F8944091FD
:10452000C9015091CA016091CB017091CC018FBF3C
:10453000CA010895CF92DF92EF92FF920F931F93DB
:104540002FB7F8944091C9015091CA016091CB01F5
:104550007091CC012FBF6A017B01EE24FF248C01F6
:1045600020E030E0C016D106E206F30620F09A0102
:10457000281B390B05C09C0120953095240F351F51
:10458000C9011F910F91FF90EF90DF90CF90089598
:104590001F920F920FB60F9211248F939F93AF9398
:1045A000BF938091C9019091CA01A091CB01B091B4
:1045B000CC010196A11DB11D8093C9019093CA0140
:1045C000A093CB01B093CC01BF91AF919F918F91FC
:1045D0000F900FBE0F901F9018950E94D111F89464
:1045E0002FEF87EA91E6215080409040E1F700C02C
:1045F000000087E090EBDC018093EA019093EB01EF
:10460000A093EC01B093ED012CE088E190E00FB6AF
:10461000F894A895809360000FBE20936000FFCFB0
:10462000CF92DF92EF92FF920F931F93CF93DF937E
:10463000C82ED12C01E010E08D2D0E94BF0A7C0114
:10464000C0E0D0E098010C2E02C0220F331F0A9464
:10465000E2F72E213F21232B29F42196CF30D105DB
:1046600089F708C06C2F7D2D80E00E94E30BC812F3
:10467000F4CF06C0D39485E0D812DECF80E001C02D
:1046800081E0DF91CF911F910F91FF90EF90DF902C
:10469000CF900895CF93C82F8CE20E9410238823D7
:1046A00021F08C2FCF910C94102380E0CF910895AE
:1046B000CF930E94AA24811102C00E948B2485EB13
:1046C00094E00E948308C5E608C00E947D098FE33C
:1046D0009CE90197F1F700C00000C150B1F78AECE6
:1046E00094E00E94830889E20E944A23811111C14B
:1046F0008AE20E944A2381110E948B2485E00E9455
:104700004A2381110E94ED220E94B5248093C501A5
:1047100087E00E944A23882399F18BE10E944A2373
:10472000882351F09091C50191FB882780F921E001
:10473000822780FB91F922C08EE00E944A238823C1
:1047400051F09091C50192FB882780F921E08227E2
:1047500080FB92F913C080E10E944A239091C50129
:10476000882341F093FB882780F921E0822780FB92
:1047700093F904C0892F809580FB90F99093C5012F
:104780008091C5010E94B9240E94C7248093DA0158
:1047900080EE0E944A23882341F08091DA01982F0D
:1047A000909590FB80F98093DA0189E30E944A2377
:1047B000882359F09091DA0191FB882780F921E054
:1047C000822780FB91F99093DA0182EE0E944A23BE
:1047D000882359F09091DA0192FB882780F921E033
:1047E000822780FB92F99093DA0186EE0E944A2399
:1047F000882359F09091DA0193FB882780F921E012
:10480000822780FB93F99093DA0183EE0E944A237A
:10481000882359F09091DA0194FB882780F921E0F0
:10482000822780FB94F99093DA0185E30E944A2362
:10483000882359F09091DA0195FB882780F921E0CF
:10484000822780FB95F99093DA0181E30E944A2345
:10485000882359F09091DA0196FB882780F921E0AE
:10486000822780FB96F99093DA0181E10E944A2326
:10487000882359F09091DA0197FB882780F921E08D
:10488000822780FB97F99093DA018091DA010E94E8
:10489000CB248091DA0187FB882780F980930D0172
:1048A00087E20E944A23C82F8EE10E944A23811189
:1048B000C2608FE10E944A238111C46080E20E949D
:1048C0004A238111C86081E20E944A238111C0619C
:1048D00082E20E944A238111C06283E20E944A233D
:1048E0008111C06484E20E944A23882311F0C068C9
:1048F00002C0CC2329F08C2F0E94C2246C2F03C04D
:104900000E94BE24682F70E080E090E0CF910C946C
:10491000851FCF9108956DEE7EEF80E090E00E94BC
:10492000B13060E082E090E00E94A33060E083E07C
:1049300090E00E94A33060E084E090E00E94A33009
:1049400060E085E090E00E94A33060E086E090E0C7
:104950000C94A33080E090E00E949D3021E08D3ED9
:104960009E4F09F020E0822F089582E090E00C94A1
:104970009530682F82E090E00C94A33083E090E0C3
:104980000C949530682F83E090E00C94A33084E081
:1049900090E00C949530682F84E090E00C94A33064
:1049A00086E090E00C949530682F86E090E00C94BF
:1049B000A3308091D50180FF0BC06091130185E089
:1049C000689FB001112475956795759567952AC004
:1049D00081FF09C06091130185E0689FB001112437
:1049E000759567951FC082FF07C06091130185E030
:1049F000689FB001112416C04091CF014423C9F033
:104A000060911201461788F72091130185E0289FD5
:104A100090011124429FC001439F900D112470E02A
:104A20000E9467306038710540F46115710539F0F6
:104A300002C065E070E0862F08958FE7089581E059
:104A400008958091D50180FF08C06091110170E048
:104A5000759567957595679521C081FF06C0609132
:104A6000110170E07595679519C082FF04C06091CF
:104A7000110170E010C08091CF018823C1F06091D6
:104A800010018617A0F790911101989FC001112481
:104A900070E00E9467306038710528F46115710577
:104AA00021F0862F08958FE7089581E0089561E051
:104AB00070E0F4CF803F21F40E94D924819504C096
:104AC000813F29F40E94D9248093D2010895823F26
:104AD00021F40E94D924819504C0833F29F40E94C7
:104AE000D9248093D1010895893F19F40E9421258A
:104AF00005C08A3F31F40E94212581958093D3011E
:104B000008958B3F21F40E942125819504C08C3F9C
:104B100029F40E9421258093D4010895843F21F433
:104B20008091D001816017C0853F21F48091D00130
:104B3000826011C0863F21F48091D00184600BC057
:104B4000873F21F48091D001886005C0883F31F40F
:104B50008091D00180618093D00108958D3F21F430
:104B60008091D50181600BC08E3F21F48091D501E9
:104B7000826005C08F3F29F48091D50184608093C5
:104B8000D5010895803F29F48091D20187FF6EC03E
:104B900007C0813F41F48091D20118160CF066C025
:104BA0001092D20163C09091D101823F19F497FF16
:104BB0005DC005C0833F31F419160CF057C0109248
:104BC000D10154C0893F31F48091D30118160CF003
:104BD0004DC006C08A3F39F48091D30187FF46C09B
:104BE0001092D30143C08B3F29F48091D40187FFF9
:104BF0003DC006C08C3F39F48091D4011816B4F53D
:104C00001092D40133C0843F21F48091D0018E7F73
:104C100005C0853F31F48091D0018D7F8093D00114
:104C200025C0863F21F48091D0018B7FF7CF873F4D
:104C300021F48091D001877FF1CF883F21F48091CA
:104C4000D0018F7EEBCF8D3F21F48091D5018E7FF7
:104C50000BC08E3F21F48091D5018D7F05C08F3F21
:104C600029F48091D5018B7F8093D5018091D1016A
:104C700081110EC08091D20181110AC08091D301AF
:104C8000811106C08091D401811102C01092CF0120
:104C900008958091C50183FF7EC081ED94E00E945C
:104CA00083088091D0011F928F9384EF94E09F93AB
:104CB0008F930E941C0989EF94E00E948308209141
:104CC000D101822F992787FD90959F932F938BEF8A
:104CD00094E09F938F930E941C098EEF94E00E94B2
:104CE00083082091D201822F992787FD90959F9369
:104CF0002F9380E095E09F938F930E941C0983E09F
:104D000095E00E9483082091D301822F992787FD87
:104D100090959F932F9385E095E09F938F930E94AA
:104D20001C0988E095E00E9483082091D401822F1D
:104D3000992787FD90959F932F938AE095E09F9305
:104D40008F930E941C098DE095E00E94830880915A
:104D5000CF011F928F9380E195E09F938F930E94E4
:104D60001C0983E195E00E9483088091D5011F9280
:104D70008F9385E195E09F938F930E941C0988E1B2
:104D800095E00E9483088DB79EB74C960FB6F894B5
:104D90009EBF0FBE8DBF80ED91E00E9443150E9423
:104DA0008D229093CE018093CD010895CF93809171
:104DB000CD019091CE010E949A224091CF014423CF
:104DC00021F02091140130E006C0209115015AE035
:104DD000259F900111248217930708F486C08091C3
:104DE000D10181110DC09091D201911109C0909112
:104DF000D301911105C09091D401992309F475C094
:104E00004F3F19F04F5F4093CF01181624F40E94D2
:104E1000D9248093D1018091D10187FF05C00E94E0
:104E2000D92481958093D1018091D201181624F460
:104E30000E94D9248093D2018091D20187FF05C0BE
:104E40000E94D92481958093D2016091D10166237B
:104E500039F1C091D201CC2319F1772767FD709504
:104E6000872F972F0E94782F23E333E343E35FE3F9
:104E70000E94DC2F0E94452F6093D1016C2F772771
:104E800067FD7095872F972F0E94782F23E333E3D8
:104E900043E35FE30E94DC2F0E94452F6093D20121
:104EA0008091D301181624F40E9421258093D30108
:104EB0008091D30187FF05C00E94212581958093B1
:104EC000D3018091D401181624F40E9421258093E7
:104ED000D4018091D40187FF05C00E9421258195CE
:104EE0008093D401CF910C944926CF910895E0EDA1
:104EF000F1E085E0DF011D928A95E9F71092CF017C
:104F00001092D50108958FE39BE00E9483088BE502
:104F10009BE00E94830888E69BE00C94830880ED68
:104F20009BE00E94830888EF9BE00E94830885E055
:104F30009CE00E94830880E29CE00E9483088BE34F
:104F40009CE00E94830883E59CE00E9483088DE634
:104F50009CE00E9483088BE89CE00E9483088BEA17
:104F60009CE00E94830880EC9CE00E94830887ED0F
:104F70009CE00E94830884EF9CE00E94830883E108
:104F80009DE00E94830883E39DE00E94830885E5FD
:104F90009DE00E9483088AE89DE00E9483081F929A
:104FA00085E08F938FE99DE09F938F930E941C096A
:104FB00082EA9DE00E9483081F9281E08F938BEA32
:104FC0009DE09F938F930E941C098EEA9DE00E94B2
:104FD00083088DB79EB708960FB6F8949EBF0FBE94
:104FE0008DBF80EB9DE00C948308833009F45AC098
:104FF00030F4813069F0823009F0E9C02EC085308C
:1050000009F49AC008F473C0863009F0E0C0B9C052
:1050100020911501862F90E0820F911D8F3F910501
:1050200020F4620F6093150103C08FEF8093150188
:1050300085EF9EE00E948308809115011F928F9357
:1050400081E09FE09F938F930E941C090F900F9027
:105050000F900F9084E09FE0B8C020911401862F3C
:1050600090E0820F911D8F3F910520F4620F6093B5
:10507000140103C08FEF8093140186E09FE00E942B
:105080008308809114011F928F9385E19FE09F9385
:105090008F930E941C090F900F900F900F9088E142
:1050A0009FE093C020911301862F90E0820F911D05
:1050B0008F3F910520F4620F6093130103C08FEFBF
:1050C000809313018AE19FE00E948308809113017D
:1050D0001F928F938AE29FE09F938F930E941C09F7
:1050E0000F900F900F900F908DE29FE06EC0209177
:1050F0001201862F90E0820F911D8F3F910520F4C1
:10510000620F6093120103C08FEF809312018FE250
:105110009FE00E948308809112011F928F9381E487
:105120009FE09F938F930E941C090F900F900F9008
:105130000F9084E49FE049C020911101862F90E0F8
:10514000820F911D8F3F910520F4620F6093110132
:1051500003C08FEF8093110186E49FE00E948308D3
:10516000809111011F928F938CE59FE09F938F9305
:105170000E941C090F900F900F900F908FE59FE0F9
:1051800024C020911001862F90E0820F911D8F3F47
:10519000910520F4620F6093100103C08FEF80939C
:1051A000100181E69FE00E948308809110011F9208
:1051B0008F9389E79FE09F938F930E941C090F9024
:1051C0000F900F900F908CE79FE00C948308089548
:1051D000833009F44EC030F4813069F0823009F038
:1051E000C5C028C0853009F482C008F461C086308B
:1051F00009F0BCC09BC080911501681720F4861B84
:105200008093150102C0109215018EE79FE00E9465
:105210008308809115011F928F938AE89FE09F93E6
:105220008F930E941C090F900F900F900F908DE8A4
:105230009FE09AC080911401681720F4861B809328
:10524000140102C0109214018FE89FE00E948308AD
:10525000809114011F928F938EE99FE09F938F930B
:105260000E941C090F900F900F900F9081EA9FE011
:105270007BC080911301681720F4861B8093130173
:1052800002C01092130183EA9FE00E94830880917C
:1052900013011F928F9383EB9FE09F938F930E9444
:1052A0001C090F900F900F900F9086EB9FE05CC051
:1052B00080911201681720F4861B8093120102C0AE
:1052C0001092120188EB9FE00E94830880911201E6
:1052D0001F928F938AEC9FE09F938F930E941C09EB
:1052E0000F900F900F900F908DEC9FE03DC080913C
:1052F0001101681720F4861B8093110102C01092DF
:1053000011018FEC9FE00E948308809111011F9290
:105310008F9385EE9FE09F938F930E941C090F90BF
:105320000F900F900F9088EE9FE01EC080911001AB
:10533000681720F4861B8093100102C010921001A0
:105340008AEE9FE00E948308809110011F928F9344
:1053500082E090E19F938F930E941C090F900F9021
:105360000F900F9085E090E10C9483080895CF93FF
:10537000C82F85E79BE00E9483086091AE01709181
:10538000AF018091B0019091B1010E94A0211F92C4
:105390008F932CE83BE03F932F930E941C098FE8EA
:1053A0009BE00E9483081F92CF9324E93BE03F9348
:1053B0002F930E941C0987E99BE00E94830861E00B
:1053C00070E080E090E004C0660F771F881F991F8F
:1053D000CA95D2F70E94851F8DB79EB708960FB663
:1053E000F8949EBF0FBE8DBFCF910C94801BCF93BE
:1053F000482F50E0FA013697E334F10508F0E1C296
:10540000EA5AFF4F0C947B308BE195E00E948308B1
:1054100083EE97E00E9483080E94BE241F928F9320
:1054200083EF97E09F938F930E941C0986EF97E08C
:105430000E9483080E94B524C82F88EF97E00E943D
:1054400083081F92CF932BE038E03F932F930E9465
:105450001C0980E198E00E94830882E198E00E94A4
:1054600083088C2F81701F928F932CE138E03F933B
:105470002F930E941C098FE198E00E94830881E22B
:1054800098E00E948308C1FB882780F91F928F93C0
:105490002BE238E03F932F930E941C098EE298E0A4
:1054A0000E94830880E398E00E948308C2FB88275B
:1054B00080F91F928F932CE338E03F932F930E9443
:1054C0001C098FE398E00E94830881E498E00E9421
:1054D0008308C3FBCC27C0F91F92CF938AE498E0DE
:1054E0009F938F930E941C098DE498E00E9483088B
:1054F0000E94C724C82F8FE498E00E9483081F925F
:10550000CF9323E638E03F932F930E941C0988E64F
:1055100098E00E9483088AE698E00E9483088C2F16
:1055200081701F928F9323E838E03F932F930E945E
:105530001C098DB79EB780960FB6F8949EBF0FBE1C
:105540008DBF86E898E00E94830888E898E00E9472
:105550008308C1FB882780F91F928F932FE938E0D9
:105560003F932F930E941C0982EA98E00E948308CF
:1055700084EA98E00E948308C2FB882780F91F9282
:105580008F9326EB38E03F932F930E941C0989EB01
:1055900098E00E9483088BEB98E00E948308C3FB8D
:1055A000882780F91F928F932DEC38E03F932F933B
:1055B0000E941C0980ED98E00E94830882ED98E02B
:1055C0000E948308C4FB882780F91F928F932CEDDB
:1055D00038E03F932F930E941C098FED98E00E94C2
:1055E000830881EE98E00E948308C5FB882780F934
:1055F0001F928F9323EF38E03F932F930E941C0953
:1056000086EF98E00E94830888EF98E00E94830864
:10561000C6FB882780F91F928F9324E139E03F93DE
:105620002F930E941C0987E199E00E94830889E179
:1056300099E00E948308C7FBCC27C0F91F92CF9343
:1056400081E299E09F938F930E941C0984E299E084
:105650000E9483080E94D024C82F86E299E00E940D
:1056600083081F92CF932DE339E03F932F930E943D
:105670001C098DB79EB780960FB6F8949EBF0FBEDB
:105680008DBF82E499E00E94830884E499E00E943F
:1056900083088C2F81701F928F932EE439E03F9303
:1056A0002F930E941C0981E599E00E94830883E5FD
:1056B00099E00E948308C6951F92CF938CE599E0EC
:1056C0009F938F930E941C098FE599E00E948308A5
:1056D0008DB79EB708960FB6F8949EBF0FBE8DBFCC
:1056E0001DC00E94ED14892B79F00E94ED14909357
:1056F000D8018093D7010E94801B80E090E00E9437
:10570000E81486E295E008C08091D7019091D80115
:105710000E94E8148FE295E00E94830881E056C160
:1057200081E699E00E9483088DE799E00E94830852
:1057300084E999E00E9483088CEA99E00E9483083A
:1057400084EC99E00E9483088EED99E00E94830822
:1057500085EF99E00E94830885E19AE00E94830822
:105760008BE29AE00E9483088CE39AE00E9483080F
:1057700084E59AE00E94830884E69AE00E94830808
:105780008EE79AE00E94830887E99AE00E948308E6
:1057900080EB9AE00E94830889EC9AE00E948308DB
:1057A00082EE9AE00E94830883E09BE00E948308D7
:1057B00085E29BE0B1CF8091C501817F8E7F809390
:1057C000C5010E9483278AE395E00E9483088FE445
:1057D00095E00E94830881E08093D601F7C00E9483
:1057E000801B83E595E00E9483089FEF23ED80E313
:1057F000915020408040E1F700C000000E94ED225F
:105800008CE695E089CF8091C50180FF09C08CE7C7
:1058100095E00E9483088091C501817F8E7F17C02B
:105820008FE895E00FC09091C50191FB882780F922
:1058300021E0822780FB91F99093C501882351F0E4
:1058400081EA95E00E9483088091C5018160809380
:10585000C50164CF8AEB95E05FCF9091C50192FBC3
:10586000882780F921E0822780FB92F99093C50177
:10587000882319F084ED95E0E5CF8FEE95E04CCFCD
:105880009091C50193FB882780F921E0822780FB56
:1058900093F99093C501882319F08BE096E0D2CF5D
:1058A00083E296E039CF8CE396E00E94830883E59B
:1058B00096E00E94830889E796E00E9483088DEBBA
:1058C00096E00E94830884EE96E00E94830889E2B5
:1058D00097E022CF8091C9019091CA01A091CB019C
:1058E000B091CC01BF93AF939F938F9384E597E0E2
:1058F0009F938F930E941C090F900F900F900F9011
:105900000F900F900BCF88E697E00E9483080E94CB
:10591000F2141F928F938EE797E09F938F930E94CC
:105920001C0980910C011F928F9388E997E09F9347
:105930008F930E941C0980914E011F928F938FEAD2
:1059400097E09F938F930E941C098DB79EB70C968A
:105950000FB6F8949EBF0FBE8DBFE0CE0E94801B95
:1059600080910D0191E0892780930D01882319F022
:1059700082EC97E0D1CE81ED97E0CECE81E890E049
:105980000E944E159FEF21EE84E091502040804010
:10599000E1F700C0000080E090E00E944E159FEF0C
:1059A00029E688E1915020408040E1F700C00000E6
:1059B000B5CE80E003C08D5101C089530E94B72944
:1059C000ADCE81EE97E00E94830880E0CF910895EC
:1059D00080E0089580E00895CF93C82F8091D6018C
:1059E000813071F020F0823009F063C14FC0A09186
:1059F0000E01B0910F018C91823209F05CC107C099
:105A0000A0910E01B0910F018C91823249F48C2F3C
:105A10000E94E82C811136C08C2F0E94F72934C0D7
:105A20008C2F0E94EA2C81112DC0C43189F028F4FA
:105A3000CB3039F0C03109F512C0C93249F0C83352
:105A4000E1F40E94832789E99BE00E9483081AC041
:105A50008DE99BE00E9483081092D6012EC10E941E
:105A60008F2781EB9BE00E9483088AEC9BE00E94D9
:105A7000830882E08093D60105C08EEC9BE00E94F3
:105A800083081BC181E090E081701AC1C83280F4A4
:105A9000CE3108F0ABC0CB30F9F020F4C73009F0BC
:105AA000EBC0D3C0C33149F1C43109F0E5C017C020
:105AB000CB3409F4BEC030F4C93289F0C83309F0E0
:105AC000DBC00AC0C13509F4B2C0C23509F4ADC0AB
:105AD000CE3409F0D1C0B3C00E948F27D2C010923B
:105AE000D9018DED9DE00E94830885EF9DE00E9425
:105AF000830881E08093D601E3C082E39EE00E94A8
:105B0000830885E59EE00E948308809115011F921D
:105B10008F938AE69EE09F938F930E941C098DE6E7
:105B20009EE00E9483088FE69EE00E948308809199
:105B300014011F928F9384E89EE09F938F930E949D
:105B40001C0987E89EE00E94830889E89EE00E9485
:105B50008308809113011F928F938BE99EE09F939E
:105B60008F930E941C098EE99EE00E94830880EAC0
:105B70009EE00E948308809112011F928F9384EB14
:105B80009EE09F938F930E941C0987EB9EE00E94EA
:105B9000830889EB9EE00E948308809111011F9287
:105BA0008F9381ED9EE09F938F930E941C0984ED5B
:105BB0009EE00E94830886ED9EE00E94830880910B
:105BC00010011F928F9380EF9EE09F938F930E940E
:105BD0001C0983EF9EE00E9483088DB79EB748960C
:105BE0000FB6F8949EBF0FBE8DBF4BC0CE51EC2FA9
:105BF000F0E0E15DFE4F80818093D90189EF9DE067
:105C00000E9483088091D9011F928F938EE09EE0BD
:105C10009F938F930E941C0981E19EE00E9483085C
:105C20000F900F900F900F902CC061E003C061E0C7
:105C300007C06AE08091D9010E94F52722C06AE07E
:105C40008091D9010E94E8281CC08EE18093150143
:105C500082E3809314018AE08093130184E18093AE
:105C6000120188E08093110188E28093100183E1A2
:105C70009EE00E94830805C088E29EE00E9483089F
:105C800016C08AE29EE00E9483088091D9011F928B
:105C90008F938CE29EE09F938F930E941C098FE26A
:105CA0009EE00E9483080F900F900F900F9081E06C
:105CB00007C01092D60180E003C080E090E0E4CEFF
:105CC000CF9108950E94AA24811102C00E948B24C2
:105CD0000E94D0248093E90180FF02C0869501C014
:105CE00080E00C94F10C8091E901982F9695292F72
:105CF00030E02F3031054CF49F5F990F8170892B74
:105D000081608093E9010E94D4248091C50180FFC5
:105D10000FC08091E90186951F928F9387E090E1F3
:105D20009F938F930E941C090F900F900F900F90DC
:105D30008091E90186950C94F10C8091E901982FEE
:105D4000969591F09158990F8170892B8093E90174
:105D50008E7F91E009F490E08091E90190FB80F959
:105D60008093E9010E94D4248091C50180FF0FC077
:105D70008091E90186951F928F938FE190E19F9327
:105D80008F930E941C090F900F900F900F9080919D
:105D9000E90186950C94F10C8091E901982F90957A
:105DA00090FB80F98093E9010E94D4248091C50181
:105DB00080FF0FC08091E90181701F928F9387E36C
:105DC00090E19F938F930E941C090F900F900F906A
:105DD0000F908091E90180FF02C0869501C080E0AC
:105DE0000C94F10C3091E901232F26952F5F2F772A
:105DF000822F90E0317040972CF4220F232B2093B8
:105E0000E90102C03093E9018091E901282F2E7F3A
:105E100091E009F490E090FB80F98093E9010E9401
:105E2000D4248091C50180FF0FC08091E90186953F
:105E30001F928F938DE490E19F938F930E941C0992
:105E40000F900F900F900F908091E90186950C9420
:105E5000F10C2091E901922F96959827990F822FA6
:105E60008170892B8093E9018E7F91E009F490E0A5
:105E70008091E90190FB80F98093E9010E94D4248C
:105E80008091E90186950C94F10C04D06894B111CD
:105E90008DC0089570D088F09F5790F0B92F992742
:105EA000B751A0F0D1F0660F771F881F991F1AF025
:105EB000BA95C9F712C0B13081F077D0B1E008953A
:105EC00074C0672F782F8827B85F39F0B93FCCF3BB
:105ED000869577956795B395D9F73EF4909580951B
:105EE000709561957F4F8F4F9F4F0895E89409C03B
:105EF00097FB3EF490958095709561957F4F8F4FFD
:105F00009F4F9923A9F0F92F96E9BB279395F69512
:105F1000879577956795B795F111F8CFFAF4BB0F90
:105F200011F460FF1BC06F5F7F4F8F4F9F4F16C0F4
:105F3000882311F096E911C0772321F09EE8872F7E
:105F4000762F05C0662371F096E8862F70E060E03A
:105F50002AF09A95660F771F881FDAF7880F9695B3
:105F6000879597F9089557FD9058440F551F59F09C
:105F70005F3F71F04795880F97FB991F61F09F3F36
:105F800079F087950895121613061406551FF2CF5F
:105F90004695F1DF08C0161617061806991FF1CFAF
:105FA00086957105610508940895E894BB276627D6
:105FB0007727CB0197F908950BD078C069D028F0E6
:105FC0006ED018F0952309F05AC05FC01124EECFAF
:105FD000CADFA0F3959FD1F3950F50E0551F629F44
:105FE000F001729FBB27F00DB11D639FAA27F00D32
:105FF000B11DAA1F649F6627B00DA11D661F829F59
:106000002227B00DA11D621F739FB00DA11D621F3D
:10601000839FA00D611D221F749F3327A00D611D5A
:10602000231F849F600D211D822F762F6A2F11243C
:106030009F5750408AF0E1F088234AF0EE0FFF1F8F
:10604000BB1F661F771F881F91505040A9F79E3FC6
:10605000510570F014C0AACF5F3FECF3983EDCF31B
:10606000869577956795B795F795E7959F5FC1F703
:10607000FE2B880F911D9695879597F9089597F9AE
:106080009F6780E870E060E008959FEF80EC0895DE
:1060900000240A9416161706180609060895002407
:1060A0000A9412161306140605060895092E039481
:1060B000000C11F4882352F0BB0F40F4BF2B11F4F5
:1060C00060FF04C06F5F7F4F8F4F9F4F089597FB16
:1060D000072E16F4009407D077FD09D00E94813076
:1060E00007FC05D03EF4909581959F4F08957095DB
:1060F00061957F4F0895EE0FFF1F0590F491E02DFD
:106100000994AA1BBB1B51E107C0AA1FBB1FA617FE
:10611000B70710F0A61BB70B881F991F5A95A9F750
:1061200080959095BC01CD010895F999FECF92BD5F
:1061300081BDF89A992780B50895A8E1B0E042E0C2
:1061400050E00C94B830262FF999FECF1FBA92BDBB
:1061500081BD20BD0FB6F894FA9AF99A0FBE019648
:1061600008950E94A330272F0C94A430DC01CB01AA
:10617000FC01F999FECF06C0F2BDE1BDF89A319657
:1061800000B40D9241505040B8F70895F894FFCFF5
:106190000540100DF40DD00D9B0D670D0101B501EB
:1061A0002808140A321E9D02B602CF02E802080334
:1061B0000604B903830363032A033F4D36203901E4
:0A61C00002030405060708090000A9
:00000001FF
